:040000000BEF00F012
:100008005F82FACF50F0FBCF51F07EED1EF074EF17
:1000180017F0700E0001856F000E0001866F65EF06
:1000280005F0250E00018C19D8B40BD06CC0D9FF8F
:100038006DC0DAFF8CC0DFFF00016C4B6D2B65EFE4
:1000480005F0000E00018B6F000E8A6F000E000194
:100058008E6F000E8D6F0ED000018D8708D00001C5
:100068008D8105D000018E8702D000018D850001A9
:100078006E4B6F2B6EC0F6FF6FC0F7FF0800F55090
:10008800200AD8B4ECD7030AD8B4ECD70E0AD8B4EF
:10009800E3D71D0AD8B4E9D700018DA702D0000123
:1000A8008D956EC0F6FF6FC0F7FF0800F550E9ECBC
:1000B80022F0D8A041D0000E00018B6F000E8A6F8D
:1000C8008AC060F08BC061F0000E0001636F0A0EF9
:1000D800626F0FEC22F060C08AF061C08BF0D00E26
:1000E8000001766FFF0E0001776F6EC0F6FF6FC0DC
:1000F800F7FF0800F5500001786F796B0001765121
:100108000001782700017751000179230001785117
:1001180000018A270001795100018B2300016E4BF1
:100128006F2B6EC0F6FF6FC0F7FF0800F550E9ECC3
:1001380022F0D8A01AD0C4D76EC0F6FF6FC0F7FF60
:100148000800F5502A0AD8A410D085C0D9FF86C067
:10015800DAFFDECF8AF0DDCF8BF0020E00018527B3
:10016800000E862300016E4B6F2B6EC0F6FF6FC02A
:10017800F7FF0800F5502E0AD8A440D000018E8D54
:1001880000016E4B6F2B6EC0F6FF6FC0F7FF0800C3
:10019800F5502A0AD8A410D085C0D9FF86C0DAFF46
:1001A800DF500001896F020E00018527000E8623AB
:1001B80000016E4B6F2B17D1000E0001896F13D011
:1001C8006EC0F6FF6FC0F7FF0800F5CF76F00001AC
:1001D80089510A0DF35000017625D00F0001896F6F
:1001E80000016E4B6F2B6EC0F6FF6FC0F7FF080063
:1001F800F550E9EC22F0D8A0F6D0E2D7000E0001C5
:10020800896FF1D000018D8D16D100018D8B000111
:100218008D8F11D185C0D9FF86C0DAFFDECF81F07E
:10022800DDCF82F0020E00018527000E8623000133
:10023800815100018211D8A406D0840E0001816F7B
:100248007F0E0001826F000E0001846F000E836F25
:1002580003D00001834B842B0001835100018125C9
:100268000001766F00018451000182210001776F3F
:1002780076C0F6FF77C0F7FFF86A070EF76403D079
:100288000800F55005D0F6CFE1FFF7CFE2FFE750C1
:100298000009D8A4DED7000189510001D8B417D0CD
:1002A80089C076F00001776B76BF7707000183512C
:1002B8000001765D0001845100017759D8B007D05C
:1002C800000189510001836F846B83BF840700019B
:1002D8008A510001835D00018B5100018459D8B017
:1002E80009D00001835100018A5F00018451000197
:1002F8008B5B05D0000E00018B6F000E8A6F00012A
:100308008DA70AD030D06CC0D9FF6DC0DAFF200E9F
:10031800DF6E00016C4B6D2B00018A07D8A08B079C
:1003280000018A29F0E100018B29D8B41CD0EBD751
:1003380081C0F6FF82C0F7FFF86A6CC0D9FF6DC0B4
:10034800DAFF070EF76403D00800F55005D0F6CFA2
:10035800E1FFF7CFE2FFE750DF6E0001814B822B10
:1003680000016C4B6D2B00018307D8A084070001A6
:100378008329DEE100018429D8A4DAD700018DB7EA
:100388000AD09FD36CC0D9FF6DC0DAFF200EDF6E94
:1003980000016C4B6D2B00018A07D8A08B07000168
:1003A8008A29F0E100018B29D8B48BD3EBD785C01B
:1003B800D9FF86C0DAFFDF5000018C6F020E000102
:1003C8008527000E86238C0E0001816F000E000128
:1003D800826F000E0001846F010E836F5CD7C00E20
:1003E80000018D1328D06EC0F6FF6FC0F7FF000123
:1003F8006E4B6F2B0800F5CF8CF000018C51000A72
:10040800D8B46ED3580AD8B400D73B0AD8B4CFD7DB
:10041800070AD8B410D00D0AD8B40DD0060AD8B43B
:10042800F1D61C0AD8B4F6D6060AD8B4D8D70D0A1D
:10043800D8B4EDD6C8D7C00E00018D150001766F6F
:10044800000E00018E150001776F00017651000142
:100458007711D8A419D085C0D9FF86C0DAFFDECFBE
:1004680087F0DDCF88F0020E00018527000E862375
:10047800000188AF16D0030E00018D130001876DAF
:10048800881FD8B0882B0DD085C0D9FF86C0DAFF69
:10049800DECF87F0DDCF88F0020E00018527000E41
:1004A8008623000189510001D8A463D00001875137
:1004B80000018811D8A45DD00001892B5AD0010E03
:1004C80000018C6F050E00018C19D8B461D00001B1
:1004D8008C51020DFD0EF324F66E7C0EF420F76E9F
:1004E8000900F5500001875D0900F55000018859A1
:1004F800D8A04ED000018C2BE5D7010E00018C6FDF
:10050800040E00018C19D8B443D000018C51020D9F
:10051800070EF324F66E7D0EF420F76E0900F550F1
:100528000001875D0900F55000018859D8A030D036
:1005380000018C2BE5D7010E00018C6F060E00011F
:100548008C19D8B425D000018C51020DF10EF3247A
:10055800F66E7C0EF420F76E0900F5500001875DF9
:100568000900F55000018859D8A012D000018C2B41
:10057800E5D700018D51C00B000AD8B4A0D7400AB6
:10058800D8B4D9D7C00AD8B4B8D7400AD8B497D7FE
:1005980000018C51800A0001766F00018951800AA0
:1005A8000001765DD8B003D089C08CF00DD0000171
:1005B8008951800A0001766F00018C51800A000180
:1005C800765DD8A08CC089F000018A5100018B119A
:1005D800D8B414D0030E00018D150001766F000EFB
:1005E80000018E150001776F000176510001771127
:1005F800D8B404D000018A07D8A08B0700018EADBB
:1006080021D0800E000189BF7F0E0001766F0001A6
:100618008A510001895D00018B51800A00017659D9
:10062800D8B00BD00001895100018A5F000E00018B
:1006380089BFFF0E00018B5B05D0000E00018B6F98
:10064800000E8A6FC40E0001766F080E0001776FE6
:100658008DC078F08EC079F00001765100017817CE
:100668000001775100017917400E0001781910E157
:10067800080E00017919D8A40BD000018A51000195
:100688008B11D8B436D000018A07D8A08B0731D097
:10069800C00E0001766F080E0001776F8DC078F0EC
:1006A8008EC079F00001765100017817000177516A
:1006B80000017917800E000178191BE1080E00016E
:1006C8007919D8A416D000018BBF0ED000018B5128
:1006D80005E1030E00018A5DD8A006D00001FE0ED8
:1006E8008A27FF0E8B2305D0000E00018B6F000EAA
:1006F8008A6F800E00018CBF7F0E0001766F0001AB
:100708008A5100018C5D00018B51800A00017659E5
:10071800D8B00BD000018C5100018A5F000E000197
:100728008CBFFF0E00018B5B05D0000E00018B6FA4
:10073800000E8A6F00018DA570D0030E00018D1583
:100748000001766F000E00018E150001776F000121
:10075800765100017711D8B40AD06CC0D9FF6DC0AA
:10076800DAFF2D0E0CD000016C4B6D2B42D000012E
:100778008DA107D06CC0D9FF6DC0DAFF200EDF6EE7
:10078800F2D7C00E0001766F080E0001776F8DC09A
:1007980078F08EC079F000017651000178170001D9
:1007A800775100017917800E0001781922E1080EAF
:1007B80000017919D8A41DD06CC0D9FF6DC0DAFF2B
:1007C800300EDF6E00016C4B6D2B00018DBB05D028
:1007D800000E00017B6F780E04D0000E00017B6FC5
:1007E800580E7A6F6CC0D9FF6DC0DAFF7AC0DFFF90
:1007F800BAD700018A5100018B11D8B43CD16CC022
:10080800D9FF6DC0DAFF300EDF6E00016C4B6D2B27
:1008180000018A07D8A08B07ECD700018A51000194
:100828008B11D8B416D000018DB713D06CC0D9FF86
:100838006DC0DAFF200EDF6E00016C4B6D2B0001DE
:100848008A07D8A08B0700018A5100018B11D8A410
:10085800EDD7030E00018D150001766F000E000123
:100868008E150001776F0001765100017711D8B419
:100878000AD06CC0D9FF6DC0DAFF2D0E0CD0000174
:100888006C4B6D2B0AD000018DA107D06CC0D9FF2D
:100898006DC0DAFF200EDF6EF2D7C00E0001766F52
:1008A800080E0001776F8DC078F08EC079F00001D6
:1008B8007651000178170001775100017917400E31
:1008C800000178190CE1080E00017919D8A407D0A5
:1008D8006CC0D9FF6DC0DAFF300EDF6EC9D0C00E14
:1008E8000001766F080E0001776F8DC078F08EC01A
:1008F80079F0000176510001781700017751000165
:100908007917800E0001781904E1080E00017919A1
:10091800D8A4B1D06CC0D9FF6DC0DAFF300EDF6E3D
:1009280000016C4B6D2B00018DBB05D0000E000142
:100938007D6F780E04D0000E00017D6F580E7C6F1D
:100948006CC0D9FF6DC0DAFF7CC0DFFF91D0000119
:100958008951020DFD0EF324F66E7C0EF420F76E1D
:100968000900F5CF62F00A00F5CF63F087C060F0A8
:1009780088C061F0CEEC1DF060C067F061C068F01F
:10098800000E00016A6F0A0E696F24EC1FF0000167
:10099800675155D087C060F088C061F00001895167
:1009A800020D070EF324F66E7D0EF420F76E090093
:1009B800F5CF62F00A00F5CF63F0CEEC1DF0000130
:1009C80060510F0B0001806F00018DBB05D0AB0E8D
:1009D80000017E6F7E0E04D09A0E00017E6F7E0E9F
:1009E80000017F6F00018051010D7EC076F07FC04D
:1009F80077F0F35000017627F4500001772376C092
:100A0800F6FF77C0F7FF0800F5CF8CF02BD087C032
:100A180060F088C061F000018951020DF10EF324E5
:100A2800F66E7C0EF420F76E0900F5CF62F00A002E
:100A3800F5CF63F0CEEC1DF000016051070B300FCD
:100A480000018C6F0FD000018D51C00B000AD8B483
:100A58007ED7400AD8B4DBD7C00AD8B49BD7400A9F
:100A6800D8B475D76CC0D9FF6DC0DAFF8CC0DFFF72
:100A780000016C4B6D2B0001890700018929D8A45E
:100A8800E2D700018DA71DD000018BBF1AD000014D
:100A98008B5104E100018A05D8A013D06CC0D9FF9E
:100AA8006DC0DAFF200EDF6E00016C4B6D2B00016C
:100AB8008A07D8A08B0700018A5100018B11D8A49E
:100AC800EDD76EC0F6FF6FC0F7FF00016E4B6F2BBE
:100AD8000800F5CF8CF000018C51D8A415EF00F078
:100AE8006CC0D9FF6DC0DAFF000EDF6E1200ECC0DB
:100AF800E9F1EDC0EAF1000E0101EC6F000EEB6FB9
:100B0800000E0101E86F000EE76FB4D2E9C1D9FF0A
:100B1800EAC1DAFFDF500101F16F0101E94BEA2B6D
:100B280097D21B0E0101F119D8A402D0010EE3D10E
:100B38002B0E0101F119D8A402D0020EDCD10D0E42
:100B48000101F119D8B405D00A0E0101F119D8A490
:100B58000AD1010130510001F05D0101315100015C
:100B6800F159D8B084D2B40E00016C6F010E0001A7
:100B78006D6F190E00016E6F7F0E00016F6FF0C070
:100B880070F0F1C071F00DEC00F0B40E0001626F6E
:100B9800010E0001636FF9EC20F029A620D0320E77
:100BA8000101426F050E0101436F3F0E0101446FC1
:100BB800550E0101456F0001FF51200F0101466FDD
:100BC800000E0101476FF2EC0BF0040EE82EFED781
:100BD80037EC10F0010EA0EC23F0F2EC0BF0000E55
:100BE8000101F06F000EEF6FF0C0EDF1F1C0EEF112
:100BF800420E0001606F010E0001616F000E0001DE
:100C0800636F000E626F000E0001656F400E646F27
:100C180045EC22F0200E0101426F1ED0EDC1D9FF34
:100C2800EEC1DAFF020E0101EF250001F66F000E9A
:100C38000101F0210001F76F420E0001F625E16E77
:100C4800010E0001F721E26EDFCFE7FF0101ED4B56
:100C5800EE2B0101EF4BF02B010130510101ED5D4D
:100C6800010131510101EE59D8A0D8D70101F45141
:100C7800D8B404D00101F405D8A417D0020E01019C
:100C8800EF250001F66F000E0101F0210001F76F5A
:100C9800420E0001F625D96E010E0001F721DA6E29
:100CA8000D0EDF6E0101EF4BF02B0101F451D8B4AA
:100CB80005D0020E0101F419D8A417D0020E0101C3
:100CC800EF250001F66F000E0101F0210001F76F1A
:100CD800420E0001F625D96E010E0001F721DA6EE9
:100CE8000A0EDF6E0101EF4BF02B0101EF51020FED
:100CF8000101436FF0C030F1F1C031F1000E2C6EEC
:100D0800F2EC0BF0040EE82EFED737EC10F037ECBF
:100D180010F029B029A621D0320E0101426F050E2C
:100D28000101436F3F0E0101446F550E0101456FEC
:100D38000001FF51400F0101466F000E0101476F8E
:100D4800F2EC0BF0100E0001F66F940EE82EFED7B1
:100D5800F62FFCD700D037EC10F0000E0101EC6F35
:100D6800010EEB6F84D1F0C0F6F0F1C0F7F000018E
:100D7800F61FF71FF64BF72B010130510001F6273C
:100D8800010131510001F7230001F7BF58D10001DB
:100D9800F75105E13D0E0001F65DD8A050D1B40E23
:100DA80000016C6F010E00016D6F860E00016E6F01
:100DB8007E0E00016F6FF0C070F0F1C071F00DECA5
:100DC80000F0B40E0001626F010E0001636FF9ECD0
:100DD80020F029A620D0320E0101426F050E010134
:100DE800436F3F0E0101446F550E0101456F00012D
:100DF800FF51200F0101466F000E0101476FF2EC11
:100E08000BF0040EE82EFED737EC10F0010EA0EC24
:100E180023F0F2EC0BF0000E0101F06F000EEF6F03
:100E2800F0C0EDF1F1C0EEF1420E0001606F010E6D
:100E38000001616F000E0001636F000E626F000E0B
:100E48000001656F400E646F45EC22F0200E010131
:100E5800426F1ED0EDC1D9FFEEC1DAFF020E0101CB
:100E6800EF250001F66F000E0101F0210001F76F78
:100E7800420E0001F625E16E010E0001F721E26E37
:100E8800DFCFE7FF0101ED4BEE2B0101EF4BF02B1C
:100E9800010130510101ED5D010131510101EE59AE
:100EA800D8A0D8D70101EF51020F0101436FF0C05C
:100EB80030F1F1C031F1000E2C6EF2EC0BF0280E7F
:100EC800E82EFED737EC10F037EC10F0000E0101D9
:100ED800EC6F010EEB6FB3D00101304B312BB6D064
:100EE80030C1D9FF31C1DAFFF1C1DFFF0101304B59
:100EF800312B2C2A98D00101406FB9D02B0E01015B
:100F0800F119D8A41CD0030E0101406F820E000114
:100F1800606F010E0001616F000E0001636F000E2B
:100F2800626F000E0001656F320E646F45EC22F0AF
:100F3800820E01012C6F010E01012D6F98D0000E59
:100F48000101406F7CD00D0E0101F119D8B405D014
:100F58000A0E0101F119D8A468D02CC1D9FF2DC1FE
:100F6800DAFF000EDF6E820E0001A36F010E000192
:100F7800A46FF4C0A5F0F5C0A6F0820E0001F66FCC
:100F8800010E0001F76F0001F61FF71FF64BF72B54
:100F980001012C510001F6250001A76F01012D5117
:100FA8000001F7210001A86F4DEC08F0A3C0E5F19E
:100FB800A4C0E6F10101E5510101E611D8A413D05E
:100FC80030C1D9FF31C1DAFF2B0EDF6E0101304B82
:100FD800312B30C1D9FF31C1DAFF2B0EDF6E010191
:100FE800304B312B20D0F4C060F0F5C061F0CDEC6F
:100FF80020F0B40E00016C6F010E00016D6F550EEC
:1010080000016E6F7F0E00016F6FF4C070F0F5C0C5
:1010180071F00DEC00F0B40E0001626F010E0001DA
:10102800636FF9EC20F0000E66D72CC1D9FF2DC1F3
:10103800DAFFF1C1DFFF01012C4B2D2B18D030C195
:10104800D9FF31C1DAFFF1C1DFFF46D72C2A0FD013
:1010580001014051000AD8B464D5010AD8B440D778
:10106800030AD8B44BD7010AD8B46DD7E8D7010121
:10107800E74BE82B0001EE510101E75D0001EF515C
:101088000101E859D8A042D5EBC1ECF0ECC1EDF074
:1010980012000001A8BF0ED00001A85105E1330ECF
:1010A8000001A75DD8A006D0000E0001A46F000EB5
:1010B800A36F1200A3C0E7F0A4C0E8F0AD0E0001D2
:1010C800606F000E0001616F000E0001636F000E7B
:1010D800626F000E0001656F320E646F45EC22F0FE
:1010E800000E0001EA6F000EE96F26D0E7C0D9FFB5
:1010F800E8C0DAFFDF500001EB6F0001E74BE82B97
:101108000D0E0001EB19D8B427D00A0E0001EB1917
:10111800D8B422D0200E0001EB19D8B41DD0AD0EE2
:101128000001E925D96E000E0001EA21DA6EEBC054
:10113800DFFF0001E94BEA2B0001A7510001E95D3F
:101148000001EA51800A0001A96F0001A851800A34
:101158000001A959D8A0CAD7F60E0001E56F010E03
:101168000001E66F200E0001EB19D8B42DD07CD019
:10117800E7C0D9FFE8C0DAFFDF500001EB6F200EAF
:101188000001EB19D8B420D00001EB51E9EC22F0B2
:10119800D8A002D0010E01D0000E0001A96F0001F5
:1011A800EB51F4EC21F0D8A002D0010E01D0000ED2
:1011B8000001A911E8A005D0E7C0E5F0E8C0E6F015
:1011C80038D00001E74BE82B0001E9510001A96F75
:1011D8000001EA510001AA6F0001E94BEA2B000166
:1011E800A7510001A95D0001AA51800A0001AB6F57
:1011F8000001A851800A0001AB59D8B01AD0B8D75D
:10120800E7C0D9FFE8C0DAFFDF500001EB6F0D0E31
:101218000001EB19D8B428D00A0E0001EB19D8B494
:1012280023D00001EB510001D8B41ED00001E74BD8
:10123800E82B0001E9510001A96F0001EA51000102
:10124800AA6F0001E94BEA2B0001A7510001A95D33
:101258000001AA51800A0001AB6F0001A851800A61
:101268000001AB59D8A0CCD7E9C0E3F0EAC0E4F05C
:10127800B40E00016C6F010E00016D6F580E000175
:101288006E6F7E0E00016F6FAD0E0001706F000E65
:101298000001716FE5C072F0E6C073F0E3C074F04E
:1012A800E4C075F00DEC00F0B40E0001626F010EA1
:1012B8000001636FF9EC20F0000E0001EA6F000EE8
:1012C800E96F0001EABF0AD00001EA5106E1640EA5
:1012D8000001E95DD8B0B3D001D0B1D0E9C0A9F020
:1012E800EAC0AAF00001D890A937AA370001D8901F
:1012F800A937AA37020E0001A927000EAA23800EDB
:101308000001A925D96E020E0001AA21DA6EDE506D
:10131800DE10D8A406D0000E0001A46F000EA36F43
:101328001200800E0001A96F020E0001AA6FD8906A
:101338000001E935D96E0001EA35DA6ED890D93660
:10134800DA360001A951D9260001AA51DA22DECFE6
:1013580060F0DDCF61F04CEC21F060C0E1F061C0DD
:10136800E2F0800E0001A96F020E0001AA6FD8906A
:101378000001E935D96E0001EA35DA6ED890D93620
:10138800DA360001A951D9260001AA51DA22DECFA6
:1013980060F0DDCF61F0A3C062F0A4C063F0E1C0EB
:1013A80064F0E2C065F0C1EC1AF000016051000180
:1013B8006111D8A43AD0A3C09BF0A4C09CF0A5C0EA
:1013C8009DF0A6C09EF0E5C09FF0E6C0A0F0E9C081
:1013D800A9F0EAC0AAF00001D890A937AA370001FD
:1013E800D890A937AA37020E0001A927000EAA2310
:1013F800800E0001A925D96E020E0001AA21DA6E1D
:1014080001D80AD00500FA6EDE50FD6EDE50FE6E81
:10141800F850FF6EFA5012009BC0DFF09CC0E0F05D
:10142800E3C0A3F0E4C0A4F012000001E94BEA2BEA
:101438000001EABF53D70001EA5101E148D7000E85
:101448000001A46F000EA36F1200000E00019A6F36
:101458000F0E1E6EA00E1D6E000E2A6E8950200BF8
:10146800896E000E8B6EF90E946E93689250DF09A8
:10147800926E040E2F6E400E0001606F030E000185
:10148800616F000E0001636F000E626F000E0001B5
:10149800656F800E646F45EC22F077D1800E2A606C
:1014A80002D080B256D1090E2F6E53D194929494E3
:1014B800020E4DD19482070E1E6ED00E1D6E010EC7
:1014C80046D182B002D0030E2F6E1D06D8A01E068C
:1014D8001D501E10D8A459D10A0E39D19492000E6D
:1014E80080B6010E236E80A60CD02A50010D400E46
:1014F800F324D96E030EF420DA6E8150FF0ADF6EF2
:101508002A2A0001FEA922D0B40E00016C6F010E38
:1015180000016D6FFD0E00016E6F7D0E00016F6F93
:101528002AC070F00001716B80CF72F00001736BFC
:1015380092CF74F00001756B0DEC00F0B40E000151
:10154800626F010E0001636FF9EC20F0000E80B8A5
:10155800010E286E0001FEA966D02350D8A41BD026
:10156800B40E00016C6F010E00016D6FFB0E0001DF
:101578006E6F7F0E00016F6F000E0001716F210EFC
:10158800706F0DEC00F0B40E0001626F010E0001E7
:10159800636FF9EC20F02850D8A423D0B40E0001D2
:1015A8006C6F010E00016D6F3D0E00016E6F7F0EB6
:1015B80000016F6F81500001956F966B0001951DBA
:1015C8000001706F0001961D0001716F0DEC00F0B5
:1015D800B40E0001626F010E0001636FF9EC20F098
:1015E80022D0B40E00016C6F010E00016D6F920ED7
:1015F80000016E6F7F0E00016F6F81500001956FC3
:10160800966B0001951D0001706F0001961D000189
:10161800716F0DEC00F0B40E0001626F010E000155
:10162800636FF9EC20F09484000E91D082A0ADD0C5
:10163800050E8DD094942850D8A418D0060E2F6E7D
:10164800E80E156E030E166E000E176E000E186E5D
:1016580029A49BD02A50010D400EF324D96E030E05
:10166800F420DA6E5EC0DFFF2A2A8FD0020E010155
:10167800F519D8A41DD7FF0E0001956FFF0E0001C4
:10168800966F2A500001976F986B000195510001E1
:1016980097270001965100019823400E00019725D5
:1016A800D96E030E00019821DA6E2B50DE18D8A4EB
:1016B800FFD6060E2F6EE80E156E030E166E000E80
:1016C800176E000E186E61D080A802D0090E2F6E1A
:1016D8001506000E165A175A185A155016101710D4
:1016E8001810D8A402D00B0E2F6E9492949429A6A9
:1016F8004CD0320E0101426F030E0101436F5F0EA1
:101708000101446FF2EC0BF040D02A50D8B419D044
:101718000001FEA916D0B40E00016C6F010E000185
:101728006D6F600E00016E6F7F0E00016F6F0DEC24
:1017380000F0B40E0001626F010E0001636FF9EC56
:1017480020F0010E00019A6F949294940B0E2F6E64
:101758001CD02F50000AD8B469D7010AD8B4B1D622
:10176800030AD8B4A7D6010AD8B4B8D6070AD8B499
:101778009DD6010AD8B45ED7030AD8B4A5D70F0AF4
:10178800D8B4E2D7030AD8B4C0D70B0E2F18D8A400
:1017980085D62A50D8B412000001FEA71200B40E54
:1017A80000016C6F010E00016D6F710E00016E6F0C
:1017B8007E0E00016F6F2AC070F00001716B9AC035
:1017C80072F00001736B0DEC00F0B40E0001626F53
:1017D800010E0001636FF9EC20F01200000E316E6B
:1017E800020E2E6E8950200B896E000E8B6E946847
:1017F80093689250DF09926E000E0101416F00015B
:10180800FEA71ED0B40E00016C6F010E00016D6FB3
:10181800F20E00016E6F7E0E00016F6F42C170F014
:101828000001716B43C172F00001736B0DEC00F0A5
:10183800B40E0001626F010E0001636FF9EC20F035
:10184800320E01014219D8A414D09296B40E0001A8
:101858006C6F010E00016D6FFF0E00016E6F7E0E42
:1018680000016F6F43C170F00001716B0DEC00F067
:1018780015D00001FEA712D0B40E00016C6F010E46
:1018880000016D6F730E00016E6F7F0E00016F6FA8
:1018980043C170F00001716B0DEC00F00001FEA770
:1018A800F8D0B40E0001626F010E0001636FF9EC0D
:1018B80020F0EFD0010EB7D0020EB5D00001FEA780
:1018C80026D0B40E00016C6F010E00016D6F8B0EF7
:1018D80000016E6F7F0E00016F6F2E50010D420EDA
:1018E800F324D96E010EF420DA6EDF5000018F6FF9
:1018F80000018F510001706F716B0DEC00F0B40E98
:101908000001626F010E0001636FF9EC20F02E50A8
:1019180000018F6F906BFF0E0001916FFF0E0001A9
:10192800926F010143510001936F946B0001915133
:1019380000019327000192510001942300018F5167
:101948000001931926E10001905100019419D8B4BF
:1019580029A21FD0320E01014219D8B41AD0929888
:101968000001FEA716D0B40E00016C6F010E000135
:101978006D6F430E00016E6F7F0E00016F6F0DECEF
:1019880000F0B40E0001626F010E0001636FF9EC04
:1019980020F02E50010D420EF324D96E010EF420D2
:1019A800DA6EDF50FF0A8A6E2E2A000E936E030E3F
:1019B8001DD0A00E156E860E166E010E176E000E47
:1019C800186E67D082B20ED01506000E165A175A36
:1019D800185A15285EE116285CE117285AE11828DC
:1019E800D8A457D0040E1FD09490050E316EE1D7BD
:1019F80082B40ED01506000E165A175A185A152812
:101A080048E1162846E1172844E11828D8A441D00F
:101A1800060E09D0936892889480010143512E5C88
:101A2800D8B01CD047D7316E34D00001FEA716D0ED
:101A3800B40E00016C6F010E00016D6FA50E000160
:101A48006E6F7F0E00016F6F0DEC00F0B40E000199
:101A5800626F010E0001636FF9EC20F0630EE3D7AB
:101A68003150000AD8B426D7010AD8B425D7030ABA
:101A7800D8B424D7010AD8B4A5D7070AD8B4B4D79C
:101A8800010AD8B4B5D7030AD8B4C4D7640AD8B4FD
:101A9800CCD7630E3118D8A4E3D7320E010142190E
:101AA800D8B492869480946893689250DF09926EB5
:101AB8000001FEA716D0B40E00016C6F010E0001E4
:101AC8006D6FF80E00016E6F7F0E00016F6F0DECE9
:101AD80000F0B40E0001626F010E0001636FF9ECB3
:101AE80020F0000E0101416F120004013205D8A454
:101AF80010D0040130511F0B0009D8A40AD00C8E55
:101B0800030E04013119D8A402D0010E01D0000E31
:101B18001F6E04013251D8A41200040130511F0B6A
:101B2800020AD8A41200040134510F0B0009D8B4DA
:101B38001200040134510F0B486E030E4860120066
:101B4800200E2118D8A412000C8E040134BF1BD01B
:101B5800040134510F0B486E4850020D0A0EF3244D
:101B6800D96E010EF420DA6EDECF4CF0DDCF4DF0E9
:101B7800040134510F0B486E4850010D1B0EF3241D
:101B8800D96E010E1AD0040134510F0B486E48501B
:101B9800020D0F0EF324D96E000EF420DA6EDECF9C
:101BA8004CF0DDCF4DF0040134510F0B486E485016
:101BB800010D180EF324D96E010EF420DA6EDF50F1
:101BC8004B6E4BB006D0FB0E4C144C6EFF0E4D14F2
:101BD80004D0040E4C104C6E4D504D6E040134BFB1
:101BE8000BD0040134510F0B486E4850020D0A0EF9
:101BF800F324D96E010E0AD0040134510F0B486E3C
:101C08004850020D0F0EF324D96E000EF420DA6E40
:101C18004CC0DEFF4DC0DDFF030E04013119D8A40E
:101C28002FD04CC0D9FF4DC0DAFFDFAE1CD0040165
:101C380034BF0BD0040134510F0B486E4850010DCE
:101C48001B0EF324D96E010E0AD0040134510F0B78
:101C5800486E4850010D180EF324D96E010EF42079
:101C6800DA6E0101DF824CC0D9FF4DC0DAFF000EE9
:101C7800DB844CC0D9FF4DC0DAFF000EDB8E1200AA
:101C8800040E4C184C6E4D504D6E4CC0D9FF4DC0D3
:101C9800DAFFDFAE1BD04CC0D9FF4DC0DAFF7F0E94
:101CA800DF164CC0D9FF4DC0DAFF000EDB8C000EEA
:101CB800416E050E406E4CC042F04DC043F0000E20
:101CC800456E020E446E51EC1DF006D04CC0D9FF93
:101CD8004DC0DAFF000EDB8C040E4C184C6E4D50D4
:101CE8004D6E4BB206D04CC0D9FF4DC0DAFFDFAE07
:101CF80031D0040134BF0BD0040134510F0B486EAE
:101D08004850010D1B0EF324D96E010E0AD00401B0
:101D180034510F0B486E4850010D180EF324D96E3C
:101D2800010EF420DA6E0101DF924CC0D9FF4DC0DC
:101D3800DAFF3B0EDF16000E416E050E406E4CC0FA
:101D480042F04DC043F0000E456E020E446E51EC59
:101D58001DF006D04CC0D9FF4DC0DAFF3B0EDF1690
:101D6800040134510F0B486E4850010D700EF324D6
:101D7800496E0F0EF4204A6E49C0D9FF4AC0DAFFF7
:101D8800FE0EDF161200200E216001D012006DB287
:101D980012000001FD51D8A46BD0400E0001606F05
:101DA800020E0001616F000E0001636F000E626F8A
:101DB800000E0001656F400E646F45EC22F0400E86
:101DC80000016B6F020E00016C6F400E00016D6F19
:101DD80030EC18F00001F86F0001F8510001FB6FBA
:101DE800FC6B0001FB510001FC11D8B441D0400E3E
:101DF8000001EC6F020E0001ED6FFBC0EEF0FCC0BD
:101E0800EFF0000E0001F06F020E0001F16FFBC051
:101E1800F2F0FCC0F3F0C00E0001F46F030E0001F5
:101E2800F56F7BEC05F0ECC0F9F0EDC0FAF00001BD
:101E3800FEA11ED0B40E00016C6F010E00016D6F83
:101E48000C0E00016E6F7F0E00016F6F0DEC00F03D
:101E5800B40E0001626F010E0001636FF9EC20F00F
:101E6800400E0001626F020E0001636FF9EC20F072
:101E780037EC10F037EC10F00001FD51D8A43BD03E
:101E88002C50D8A438D0000E2A6E29EC0AF02A501B
:101E9800D8B431D00001FD51D8A42DD0400E000196
:101EA800606F030E0001616F2AC062F026EC23F018
:101EB800000E2A6E0001FEA31ED0B40E00016C6F46
:101EC800010E00016D6FCA0E00016E6F7E0E0001DB
:101ED8006F6F0DEC00F0B40E0001626F010E00018F
:101EE800636FF9EC20F0400E0001626F030E0001F1
:101EF800636FF9EC20F037EC10F01200A09A000E96
:101F08006A6E000E686E000E706E710E0001606FD2
:101F18000F0E0001616F000E0001636F000E626F0B
:101F2800000E0001656F020E646F45EC22F0160E7C
:101F38006F6E9F0E6B6E7B0E696E000E0001686FF0
:101F48000B0E0001686501D010D000016851040D26
:101F5800000EF324D96E040EF420DA6EDE6ADE6A0F
:101F6800DE6ADD6A0001682BEBD76D8C000E6E6EA1
:101F78006D986D9C6896000E0C6E000E046E000E37
:101F8800066E000E056E68B6F5D7010E0101396FB1
:101F9800010E01013A6F000E0101376F000E0101B9
:101FA800386F000E0101366F000E0001686F020ED7
:101FB8000001686501D033D000016851020D0F0E91
:101FC800F324D96E000EF420DA6E000EDE6E000ED9
:101FD800DD6E00016851020D0A0EF324D96E010E60
:101FE800F420DA6E000EDE6E000EDD6E0001685120
:101FF800010D180EF324D96E010EF420DA6E000ECE
:10200800DF6E00016851010D1B0EF324D96E010E1D
:10201800F420DA6E000EDF6E0001682BC8D7080EB8
:102028000F6E040E106E160E706E040E0401036F10
:10203800300E026F080E0401016F040E0401006FD8
:102048000401008F000E326E000E0101146F000EA5
:10205800156F000E166F000E176F000E01013B6F13
:10206800000E216E1200A09A0101265101012711CC
:10207800D8B409D026C1D9FF27C1DAFF0101DFAEE4
:1020880002D0A08A1200030E0001FD19D8A403D0C3
:10209800000E0001FD6F0001FD51D8A402D0A08AF6
:1020A8001200020E0001FD19D8A417D0010E00017C
:1020B800606F000E0001616F000E0001626F000E7C
:1020C8000001636F020E86EC11F060C026F161C05A
:1020D80027F1030E0001FD6F6DD00001FD05D8A4A6
:1020E80069D0400E256404D0400E00016C6F02D008
:1020F80025C06CF000016C5100082524256E000EE7
:1021080001011E6F050E01011F6F6CC06BF001010C
:102118003D51D8B413D02AD021C1D9FF22C1DAFF4A
:102128001EC1E1FF1FC1E2FFDFCFE7FF01011E4B28
:102138001F2B0101214B222B00016B0700016B5162
:102148000001D8B418D0E8D721C1D9FF22C1DAFFDD
:102158001EC1E1FF1FC1E2FFDFCFE7FF01011E4BF8
:102168001F2B0101214B222B00016B0700016B5132
:102178000001D8A4E9D72550D8A40AD0400E000100
:102188006C19D8A402D0020E01D0030E0001FD6F15
:10219800010E0001606F000E0001616F050E000165
:1021A800626F6CC063F0020E86EC11F060C026F11D
:1021B80061C027F1A08A1200A09A000E6A6E000E74
:1021C800686E000E706E710E346E0F0E356E000E56
:1021D800376E000E366E000E396E020E386EBEEC8B
:1021E80022F0160E6F6E9F0E6B6E7B0E696E000EE0
:1021F8003C6E0B0E3C6401D00ED03C50040D000E1A
:10220800F324D96E040EF420DA6EDE6ADE6ADE6A22
:10221800DD6A3C2AEED76D8C000E6E6E6D986D9C53
:102228006896000E0C6E000E046E000E066E000E10
:10223800056E68B6F5D7010E0101396F010E01016F
:102248003A6F000E0101376F000E0101386F000E62
:102258000101366F000E3C6E020E3C6401D02ED098
:102268003C50020D0F0EF324D96E000EF420DA6EE6
:10227800000EDE6E000EDD6E3C50020D0A0EF324D9
:10228800D96E010EF420DA6E000EDE6E000EDD6EE1
:102298003C50010D180EF324D96E010EF420DA6EAD
:1022A800000EDF6E3C50010D1B0EF324D96E010E9B
:1022B800F420DA6E000EDF6E3C2ACED7080E0F6EC1
:1022C800040E106E160E706E040E0401036F300EAD
:1022D800026F080E0401016F040E0401006F04016F
:1022E800008F000E326E000E0101146F000E156F84
:1022F800000E166F000E176F000E01013B6F000EE7
:10230800216E12000001686F000160510001D8B40D
:1023180008D000016851020D0F0EF324D96E000E8B
:1023280007D000016851020D0A0EF324D96E010E80
:10233800F420DA6EDECF69F0DDCF6AF00001695172
:1023480000016A11D8A407D0000E0001606F000ECA
:102358000001616F1200000120EE02F06951D926D8
:102368006A51DA2261C0DEFF62C0DDFF000120EEA3
:1023780001F06951D9266A51DA2263C0DFFF69C0CA
:10238800D9FF6AC0DAFF400EDF1669C0D9FF6AC0FC
:10239800DAFF000EDB8669C0D9FF6AC0DAFF000EDB
:1023A800DB8E000160510001D8B41ED000016851D5
:1023B800020D0F0EF324D96E000EF420DA6EDECF74
:1023C80064F0DDCF65F0040E000164190001666F4A
:1023D800000165510001676F00016851020D0F0E81
:1023E800F324D96E000E1DD000016851020D0A0EAB
:1023F800F324D96E010EF420DA6EDECF64F0DDCF5F
:1024080065F0040E000164190001666F0001655152
:102418000001676F00016851020D0A0EF324D96E9E
:10242800010EF420DA6E66C0DEFF67C0DDFF69C00A
:1024380060F06AC061F012002104D8B46DBA06D009
:10244800000E686E69806988020E216E68B469A4FE
:1024580003D068942AEC22F06DA202D0A19A12004F
:1024680068B069A006D0E0EC10F0A08A040E216ED6
:10247800689068B869A802D08FEC22F068AC1AD0CE
:1024880069AC0ED0000E416E730E406E000E426EA7
:10249800000E436E000E456E010E446E51EC1DF0A9
:1024A800689C12EC23F02250D8A422062250D8B4FB
:1024B800A6EC16F068BA69AA02D095EC21F068B2C9
:1024C80069A20FD07F0E416E4068000E426E000E6A
:1024D800436E000E456E010E446E51EC1DF0000E69
:1024E8006A6E040E216002D0A19A120069A639D042
:1024F800000E4F6E030E4F6401D033D068A631D062
:102508006CCF33F03330E832E8320F0B276E689621
:1025180033B407D02750010D1B0EF324D96E010EDA
:1025280006D02750010D180EF324D96E010EF420A1
:10253800DA6E0101DF702750D8A403D00CEC1BF031
:102548000ED0000E416E720E406E330E426E000EBB
:10255800436E000E456E000E446E51EC1DF04F2A7E
:10256800C9D7A19A1200800E04013019D8A412000C
:10257800C00E0C6E7CD0C20E096E7D0E0A6E000E67
:102588000E6E120E0D6E120004013251D8A43ED008
:1025980004013251020D150EF324F66E7D0EF4205F
:1025A800F76E0900F5CF09F00A00F5CF0AF0020E20
:1025B8000924346E000E0A20356E34C0F6FF35C08B
:1025C800F7FFF86A070EF76403D00800F55005D046
:1025D800F6CFE1FFF7CFE2FFE7500D6E030E0924B7
:1025E800346E000E0A20356E34C0F6FF35C0F7FF92
:1025F800F86A070EF76403D00800F55005D0F6CF47
:10260800E1FFF7CFE2FFE7500E6E1200000E0C6EEE
:102618001200030E0401326124D004013251020D6C
:102628000F0EF324F66E7D0EF420F76E0900F5CF39
:1026380009F00A00F5CF0AF009C0F6FF0AC0F7FF53
:10264800F86A070EF76403D00800F55005D0F6CFF6
:10265800E1FFF7CFE2FFE750346E34500D6E0E6A9B
:102668001200000E0C6E1200000E0C6E1200040117
:102678003351010AD8B47FD7030AD8B485D7010AE1
:10268800D8B4C7D7F1D720EE01F01950D9261A507F
:10269800DA22DF50356E3550055C000E0658D8A09A
:1026A80005C035F03550055E000E065A000E346E32
:1026B80011D03450010D380EF324D96E040EF420D5
:1026C800DA6E01C0E1FF02C0E2FFDFCFE7FF014A97
:1026D800022A342A3550345CD8A0EBD705500610AE
:1026E800D8B432D020EE01F01B50D9261C50DA2283
:1026F800080EDF6E20EE02F01B50D9261C50DA229D
:10270800380EDE6E040EDD6E19C0D9FF1AC0DAFF6E
:10271800DFBC0DD01BC0D9FF1CC0DAFF480EDF6E2E
:102728001BC0D9FF1CC0DAFF000EDB8E12001BC0D5
:10273800D9FF1CC0DAFF080EDF6E1BC0D9FF1CC012
:10274800DAFF000EDB8E120020EE01F01B50D926B6
:102758001C50DA22080EDF6E20EE02F01B50D9263C
:102768001C50DA22300EDE6E040EDD6E1BC0D9FF5F
:102778001CC0DAFF040EDF6E1BC0D9FF1CC0DAFFD5
:10278800000EDB8E049E2050D8A41200A6EC16F092
:102798001200FFC0A1F00001A26B9DC0D9FF9EC02E
:1027A800DAFF000EDF6EF60E00019F1905E1010E3B
:1027B8000001A019D8B40AD09FC066F0A0C067F085
:1027C80052EC15F066C0A1F067C0A2F0320E01010C
:1027D800426F060E0101436F3F0E0101446F350E33
:1027E8000101456F180E0101466F0001A151400F0C
:1027F8000101476FF2EC0BF029EC0AF02A50D8B42B
:102808002CD09DC06CF09EC06DF0C40E00016E6FA0
:102818007F0E00016F6F40C370F00001716B0DEC0B
:1028280000F0000E2A6EB40E00016C6F010E00015C
:102838006D6F3F0E00016E6F7E0E00016F6F40C31B
:1028480070F00001716B0DEC00F0B40E0001626FC6
:10285800010E0001636FF9EC20F0320E0101426FA6
:10286800050E0101436F190E0101446F5F0E01014E
:10287800456F3F0E0101466F000E0101476FF2ECF4
:102888000BF09DC0D9FF9EC0DAFF000EDF6E000E70
:1028980000019C6F010E9B6F12003C6E3450D8B43F
:1028A80007D03C50020D0F0EF324D96E000E06D04F
:1028B8003C50020D0A0EF324D96E010EF420DA6E94
:1028C800DECF3DF0DDCF3EF03D503E10D8A405D020
:1028D800000E346E000E356E120020EE02F03D50F0
:1028E800D9263E50DA2235C0DEFF36C0DDFF20EEA5
:1028F80001F03D50D9263E50DA2237C0DFFF3DC0F7
:10290800D9FF3EC0DAFF400EDF163DC0D9FF3EC0FA
:10291800DAFF000EDB863DC0D9FF3EC0DAFF000EAD
:10292800DB8E3450D8B418D03C50020D0F0EF3246F
:10293800D96E000EF420DA6EDECF38F0DDCF39F034
:10294800040E38183A6E39503B6E3C50020D0F0E8B
:10295800F324D96E000E17D03C50020D0A0EF32452
:10296800D96E010EF420DA6EDECF38F0DDCF39F003
:10297800040E38183A6E39503B6E3C50020D0A0E60
:10298800F324D96E010EF420DA6E3AC0DEFF3BC0A4
:10299800DDFF3DC034F03EC035F012006D980CBE2E
:1029A8003BD004AE0ED0020E266E01013851D8B4C9
:1029B800D8EC19F0000E01013A6F000E0101396FD1
:1029C800120020EE01F01B50D9261C50DA22080E06
:1029D800DF6E20EE02F01B50D9261C50DA22300E92
:1029E800DE6E040EDD6E1BC0D9FF1CC0DAFF0C0EB4
:1029F800DF6E1BC0D9FF1CC0DAFF000EDB8E0FC0D4
:102A0800D9FF10C0DAFF040EDF6E0FC0D9FF10C067
:102A1800DAFF000EDB8E1200040130AF13D0010E76
:102A2800266E01013751D8B4D8EC19F0000E010117
:102A38003A6F000E0101396F2050D8A41200A6EC9D
:102A480016F01200020E266E20EE01F01B50D92659
:102A58001C50DA22080EDF6E20EE02F01B50D92639
:102A68001C50DA22300EDE6E040EDD6E1BC0D9FF5C
:102A78001CC0DAFF040EDF6E1BC0D9FF1CC0DAFFD2
:102A8800000EDB8E000E01013A6F000E0101396F56
:102A98002050D8A41200A6EC16F0120003D00001B2
:102AA800664B672B66C0D9FF67C0DAFF200EDE18B9
:102AB800D8B4F5D766C0D9FF67C0DAFF090EDE18AB
:102AC800D8B4EDD7000E00016C6F000E6B6F000ECE
:102AD80000016A6F66C0D9FF67C0DAFF2D0EDE18E5
:102AE800D8A403D000016A2B2ED066C0D9FF67C0D6
:102AF800DAFF2B0EDE18D8A429D025D06BC060F0E1
:102B08006CC061F0000E0001636F0A0E626F0FEC7B
:102B180022F066C0D9FF67C0DAFFDF500001686F96
:102B2800696B0001605100016827000161510001D3
:102B38006923D00E0001682500016B6FFF0E0001AC
:102B4800692100016C6F0001664B672B66C0D9FFD5
:102B580067C0DAFFDF50E9EC22F0D8B0CFD7000128
:102B68006A510001D8B40ED06BC068F06CC069F02F
:102B78000001681F691F684B692B68C066F069C04F
:102B880067F012006BC066F06CC067F012000C8E24
:102B9800710E346E0F0E356E000E376E000E366EE7
:102BA800000E396E020E386EBEEC22F0000E346E46
:102BB800040E356E000E376E000E366E000E396E3E
:102BC800300E386EBEEC22F06D8C000E486E020E90
:102BD800486401D016D04850010D180EF324D96E60
:102BE800010EF420DA6E000EDF6E4850010D1B0E48
:102BF800F324D96E010EF420DA6E000EDF6E482A37
:102C0800E6D7E30E346E010E356E000E376E000EF9
:102C1800366E000E396E020E386EBEEC22F06D9CD8
:102C2800080E0F6E040E106E000E196E040E1A6E4A
:102C380019C01BF01AC01CF032C432F03250D8A4AC
:102C480003D0100E216E1200000E416E010E406E70
:102C5800320E426E000E436E000E456E010E446E3B
:102C680051EC1DF0200E216E120004013039E832BB
:102C7800030B0009D8A4120043D00C8E080E216E55
:102C88001200B7EC12F01200CBEC15F01200320E65
:102C9800096E000E0A6E0C80010E0D6E0C8E12006D
:102CA80032EC19F0120079EC0DF0120004013451E5
:102CB800010DE30EF324096E010EF4200A6E0C8058
:102CC800010E0D6E0C8E12000C8E04013451010D94
:102CD800E30EF324D96E010EF420DA6E32C4DFFF5E
:102CE8001200000E416E020E406E000E426E000E83
:102CF800436E000E456E000E446E51EC1DF012003E
:102D080004013151000AD8B4CBD7010AD8B4CBD7C3
:102D1800020AD8B4C8D7060AD8B4AFD7030AD8B4B9
:102D2800B0D7010AD8B4DDD70F0AD8B4B0D7010A92
:102D3800D8B4AAD7030AD8B4B9D7010AD8B4C4D723
:102D4800070A120001013951D8A41200010E01012D
:102D5800396F01013A51D8A41200010E01013A6FEE
:102D6800020E2618D8A415D020EE01F00F50D9264F
:102D78001050DA22000EDF6E0FC0D9FF10C0DAFF44
:102D8800480EDF6E0FC0D9FF10C0DAFF000EDB8ED1
:102D980012002604D8A41200000E0101356F20EE9F
:102DA80001F01950D9261A50DA22080EDF6E20EEEB
:102DB80002F01950D9261A50DA22300EDE6E040EAF
:102DC800DD6E19C0D9FF1AC0DAFF040EDF6E19C014
:102DD800D9FF1AC0DAFF000EDB8E010E0101356F34
:102DE80020EE01F01B50D9261C50DA22080EDF6EA7
:102DF80020EE02F01B50D9261C50DA22300EDE6E6F
:102E0800040EDD6E1BC0D9FF1CC0DAFF800EDF6E1A
:102E18001200080E346E0E5010E1080E0D5CD8B08A
:102E28000CD00DC034F03050D8A402D0010E04D01C
:102E38003004D8A402D0020E306E34500D5E000E5D
:102E48000E5A20EE01F00F50D9261050DA2234C065
:102E5800DFFF380E0101326F040E0101336F0CA041
:102E68001CD03AD009C0F6FF0AC0F7FFF86A32C191
:102E7800D9FF33C1DAFF070EF76403D00800F55015
:102E880005D0F6CFE1FFF7CFE2FFE750DF6E094A42
:102E98000A2A0101324B332B34063450D8B41200BD
:102EA800E1D709C0F6FF0AC0F7FFF86A32C1D9FFB7
:102EB80033C1DAFF070EF76403D00800F55005D0D8
:102EC800F6CFE1FFF7CFE2FFE750DF6E094A0A2AA3
:102ED8000101324B332B34063450D8B41200E1D7F9
:102EE800420EF66E410EF76E000EF86E02EE80F09E
:102EF80010EE58F00900F5CFEEFFE550E150FAE189
:102F0800820EF66E470EF76E000EF86E01EEF2F0C6
:102F180010EE09F00900F5CFEEFFE550E150FAE1B7
:102F28009F0EF66E470EF76E000EF86E0900F5CF8D
:102F3800FFF09E0EF66E470EF76E000EF86E090053
:102F4800F5CF5EF003EE00F011EE00F0EE6AE5500A
:102F5800E150FCE1E250FAE102EE00F0800EEE6A88
:102F6800E806FDE101EE00F0E50EEE6AE806FDE197
:102F780004EE40F0800EEE6AE806FDE10001FE6B0B
:102F8800FD6B00EE01F0330EEE6AE806FDE15F909E
:102F98005F92000EF86E0001EEEF1EF00FC0D9FF31
:102FA80010C0DAFF000EDFBC010E356E040E0F18DC
:102FB8000F6E1050106E080E2118D8A40BD0040103
:102FC80032517F0B6E6E6E50D8B402D0100E01D005
:102FD800040E216E2604D8A43AD020EE02F00F5039
:102FE800D9261050DA22380EDE6E040EDD6E0DEC96
:102FF80017F0020E3018D8A40DD00FC0D9FF10C09A
:10300800DAFF040EDF6E0FC0D9FF10C0DAFF000E22
:10301800DB8E12003550D8A40DD00FC0D9FF10C0D8
:10302800DAFF480EDF6E0FC0D9FF10C0DAFF000EBE
:10303800DB8E12000FC0D9FF10C0DAFF080EDF6E5A
:103048000FC0D9FF10C0DAFF000EDB8E120004BEDD
:10305800049E000E266E1200000E246E01012851F7
:1030680001012911D8B407D028C1D9FF29C1DAFF35
:103078000101DFBE46D0010120EE01F02851D9261A
:103088002951DA2200016D51DE5CD8B00AD0010165
:1030980020EE01F02851D9262951DA22DF5000010B
:1030A8006D6F000E246E15D02450010D400EF324D0
:1030B800D96E050EF420DA6E2450010DF35000018C
:1030C8006B25E16EF45000016C21E26EDFCFE7FF63
:1030D800242A00016D51245CD8A0E6D7000E000117
:1030E800606F400E0001616F050E0001626F400EB7
:1030F8000001636F020E86EC11F060C028F161C018
:1031080029F124501200040130511F0BE806D8A4FD
:10311800120004013039E832030BE806D8A4120083
:1031280004013451D8B433D004013405D8A41200B2
:103138002ED0D40E096E010E0A6E000E0E6E080E09
:103148000D6E0C800C8E1200D40E096E010E0A6EE4
:103158000C8E120036C405F037C406F0DC0E016E82
:10316800010E026E000E076E000E086E048E12002D
:10317800DC0E096E010E0A6E000E0E6E070E0D6E45
:10318800C10E0C6E120032C43EF10C8E1200040106
:103198003151000AD8B4CDD7010AD8B4D5D7210AFD
:1031A800D8B4D8D7010AD8B4E3D7030AD8A41200F0
:1031B800EAD7F60E00019F1907E1010E0001A019D8
:1031C800D8A402D0000E26D0D80E0001606F7F0E62
:1031D8000001616F9FC062F0A0C063F0000E0001A3
:1031E800656F030E646FC1EC1AF0000160510001B5
:1031F8006111D8A402D0010E0DD09FC066F0A0C006
:1032080067F052EC15F0000166512B6E2B50D8B4C4
:1032180003D0020E0101F56F320E0101426F050E57
:103228000101436F3F0E0101446F550E0101456FC7
:103238000001FF51400F0101466F000E0101476F69
:10324800F2EC0BF09DC0D9FF9EC0DAFF000EDF6ED6
:10325800000E00019C6F010E9B6F1200000E04010E
:10326800386F000E0401396F38D00C8E1F04D8A4B3
:1032780040D0040138833DD00C8E3BD00C8E040125
:1032880034BF0BD0040134510F0B346E3450020D8F
:103298000A0EF324D96E010E0AD0040134510F0B23
:1032A800346E3450020D0F0EF324D96E000EF42044
:1032B800DA6EDECF35F0DDCF36F035C0D9FF36C057
:1032C800DAFFDFAE16D035C0D9FF36C0DAFFDFA48B
:1032D80010D0010E0401386F0CD0040130511F0BBF
:1032E800000AD8B4C2D7010AD8B4C6D7030AD8B4DA
:1032F800C5D70CAE1200380E096E040E0A6E0C808B
:10330800020E0D6E1200B40E00016C6F010E00016A
:103318006D6FD80E00016E6F7E0E00016F6F0DECA1
:1033280000F0B40E0001626F010E0001636FF9EC4A
:1033380020F0320E0101426F060E0101436F3F0E6D
:103348000101446F550E0101456F0001FF51200F27
:103358000101466F040E0101476F000E0101486F1D
:10336800F2EC0BF09DC0D9FF9EC0DAFF000EDF6EB5
:10337800B40E00016C6F010E00016D6FBC0E0001F0
:103388006E6F7E0E00016F6F0DEC00F0B40E000141
:10339800626F010E0001636FF9EC20F0000E00016E
:1033A8009C6F010E9B6F1200000E0101376F000E1B
:1033B8000101386F020E2618D8A41FD020EE01F0A4
:1033C8001B50D9261C50DA22080EDF6E20EE02F0C0
:1033D8001B50D9261C50DA22380EDE6E040EDD6E24
:1033E8001BC0D9FF1CC0DAFF480EDF6E1BC0D9FF17
:1033F8001CC0DAFF000EDB8E12000D500401365D92
:103408000E5004013759D8B004D036C40DF037C473
:103418000EF00DEC17F020EE02F00F50D9261050E8
:10342800DA22380EDE6E040EDD6E0FC0D9FF10C032
:10343800DAFF480EDF6E0FC0D9FF10C0DAFF000EAA
:10344800DB8E12006DA243D0010ECEEC23F01200E9
:103458000101240501012511D8A404D0010ECDECE9
:1034680023F03AD04B0E0101241901012511D8A4EB
:1034780004D0010ECEEC23F02FD00101255105E137
:10348800970E0101245DD8A027D0000E0101256FF9
:10349800000E246F21D00101240501012511D8A4B3
:1034A80004D0010ECDEC23F017D0320E01012419FF
:1034B80001012511D8A404D0010ECEEC23F00CD0C4
:1034C800B70E0101245D030E01012559DCD72150F7
:1034D800200AD8B4BDD7DFD70101244B252B120011
:1034E800000E0001A26F000EA16FF60E00019F19D9
:1034F8001EE1010E0001A019D8A419D029A602D0F6
:10350800010E01D0000E0001A16FA26B9DC06CF0EE
:103518009EC06DF0C40E00016E6F7F0E00016F6FCC
:10352800A1C070F0A2C071F00DEC00F020D09FC0D7
:1035380066F0A0C067F052EC15F066C0A1F067C055
:10354800A2F00001A1050001A211D8A404D02950BD
:103558000809296E06D02950F70B296E000EA0EC39
:1035680023F09DC0D9FF9EC0DAFF000EDF6E000E6B
:1035780000019C6F010E9B6F120039D060C0F6FFEE
:1035880061C0F7FF0800F5500009D8B40DD062C03B
:10359800D9FF63C0DAFF60C0F6FF61C0F7FFDE50F5
:1035A8000900F518D8B41DD062C0D9FF63C0DAFF8E
:1035B800DF500001666F676B0001661F671F664B6F
:1035C800672B60C0F6FF61C0F7FF0800F5500001E7
:1035D80066250001606F000E000167210001616F20
:1035E80012000001604B612B0001624B632B00014C
:1035F8006407D8A0650700016429C0E100016529B6
:10360800D8A4BCD7000E0001616F000E606F1200D5
:103618002D0E226E33C04EF0FD0E4E16D8A43BD0B0
:1036280033C04EF0D8904E323F0E4E164E50040D19
:10363800000EF324196E040EF4201A6E19C01BF044
:103648001AC01CF0040E1B181B6E1C501C6E19C0EF
:10365800D9FF1AC0DAFFDF30E8320F0B0D0AD8A401
:1036680017D0300E346E040E356E20EE02F019506D
:10367800D9261A50DA22DECF36F0DDCF37F0000E29
:10368800396E080E386EB6EC21F057EC1BF01200BC
:1036980015EC20F012003350FD0B040AD8A41200D8
:1036A800D2EC17F01200000E306E000E206E000EE5
:1036B8000101376F000E0101386F000E0101356FEF
:1036C800000E266E0FC0D9FF10C0DAFF7F0EDF167E
:1036D800040E0F180F6E1050106E0FC0D9FF10C0D7
:1036E800DAFF7F0EDF16040E0F180F6E1050106EE3
:1036F8001BC0D9FF1CC0DAFF7F0EDF16000E0C6E50
:10370800000E0E6E000E0D6E000E046E000E066E9C
:10371800000E056E39EC16F0000E416E030E406E79
:10372800000E426E000E436E000E456E000E446E93
:1037380051EC1DF0D2EC14F01200396E000E3A6E06
:10374800040E3B6E3450356E366AD89035363636B0
:103758003950376E386AD89037363836D890373679
:1037680038363550372636503822D89037363836DE
:10377800D8903736383637503A2638503B223AC038
:10378800D9FF3BC0DAFFDF9E3450D8A407D03950A8
:10379800020D0A0EF324D96E010E06D03950020D1F
:1037A8000F0EF324D96E000EF420DA6E3AC0DEFF55
:1037B8003BC0DDFF3AC0D9FF3BC0DAFFDF9C20EEFB
:1037C80004F03A50D9263B50DA22DF8C1200000E62
:1037D8000001A26F000EA16FF60E00019F191EE1F5
:1037E800010E0001A019D8A419D029A802D0010EF1
:1037F80001D0000E0001A16FA26B9DC06CF09EC0AD
:103808006DF0C40E00016E6F7F0E00016F6FA1C0D6
:1038180070F0A2C071F00DEC00F01CD09FC066F0F3
:10382800A0C067F052EC15F066C0A1F067C0A2F026
:103838000001A1050001A211D8A403D02950100944
:1038480002D02950EF0B296E9DC0D9FF9EC0DAFF28
:10385800000EDF6E000E00019C6F010E9B6F1200C0
:10386800000E0001A26F000EA16FF60E00019F1955
:103878001EE1010E0001A019D8A419D029A402D074
:10388800010E01D0000E0001A16FA26B9DC06CF06B
:103898009EC06DF0C40E00016E6F7F0E00016F6F49
:1038A800A1C070F0A2C071F00DEC00F01CD09FC058
:1038B80066F0A0C067F052EC15F066C0A1F067C0D2
:1038C800A2F00001A1050001A211D8A403D029503B
:1038D800040902D02950FB0B296E9DC0D9FF9EC058
:1038E800DAFF000EDF6E000E00019C6F010E9B6F69
:1038F8001200000E0001A26F000EA16FF60E00016B
:103908009F191EE1010E0001A019D8A419D029A2FF
:1039180002D0010E01D0000E0001A16FA26B9DC064
:103928006CF09EC06DF0C40E00016E6F7F0E00013A
:103938006F6FA1C070F0A2C071F00DEC00F01CD048
:103948009FC066F0A0C067F052EC15F066C0A1F009
:1039580067C0A2F00001A1050001A211D8A403D0FC
:103968002950020902D02950FD0B296E9DC0D9FFAC
:103978009EC0DAFF000EDF6E000E00019C6F010E84
:103988009B6F1200000E0001A26F000EA16FF60ED1
:1039980000019F191EE1010E0001A019D8A419D039
:1039A80029A002D0010E01D0000E0001A16FA26B68
:1039B8009DC06CF09EC06DF0C40E00016E6F7F0E4E
:1039C80000016F6FA1C070F0A2C071F00DEC00F0A3
:1039D8001CD09FC066F0A0C067F052EC15F066C01E
:1039E800A1F067C0A2F00001A1050001A211D8A4AE
:1039F80003D02950010902D02950FE0B296E9DC021
:103A0800D9FF9EC0DAFF000EDF6E000E00019C6F2A
:103A1800010E9B6F1200FFC0A1F00001A26B9DC0B8
:103A2800D9FF9EC0DAFF000EDF6EF60E00019F1967
:103A380005E1010E0001A019D8B40AD09FC066F0B4
:103A4800A0C067F052EC15F066C0A1F067C0A2F004
:103A5800320E0101426F060E0101436F3F0E010154
:103A6800446F550E0101456F0001A151200F01015E
:103A7800466F080E0101476F000E0101486FF2EC16
:103A88000BF09DC0D9FF9EC0DAFF000EDF6E000E5E
:103A980000019C6F010E9B6F120017D026EC1AF0E4
:103AA800120026EC1AF0010E4BEC23F0120026EC63
:103AB8001AF0020E4BEC23F01200B7EC1EF0C6EC25
:103AC80023F0120087EC18F0120040C046F041C005
:103AD80047F04750000AD8B404D07F0AD8A412008F
:103AE8001AD04650010AD8B4E8D7030AD8B412004D
:103AF800010AD8B4E7D7060AD8B41200770AD8B4AE
:103B08001200010AD8B4CAD7070AD8B4D0D7010A14
:103B1800D8A41200C6D74650FF0A1200E50E0001CD
:103B2800626F7E0E0001636FF9EC20F00F0EC11278
:103B3800200E896E000E8B6E946893689268928A44
:103B4800C70ED56EF294000E2A6E000E2C6E000E73
:103B58002D6E0BD02D50010D400EF324D96E030E9F
:103B6800F420DA6E000EDF6E2D2A7F0E2D64F2D758
:103B7800000E2D6E0BD02D50010D420EF324D96E80
:103B8800010EF420DA6E000EDF6E2D2A3F0E2D6432
:103B9800F2D71200000E0001656F000E646F00017D
:103BA800625100016311D8B42CD0010E0001666F78
:103BB80006D00001D890623763370001662B0001F8
:103BC80063AFF7D70001D8906437653700016251B9
:103BD8000001605D0001635100016159D8A00AD05D
:103BE800000162510001605F000163510001615BE7
:103BF800000164810001D890633362330001662FAD
:103C0800E1D764C060F065C061F01200000E0001E9
:103C1800606F020E0001616F000E0001636F000EFD
:103C2800626F000E0001656F400E646F45EC22F074
:103C3800000E0101406F090E296E000E0101F46F9C
:103C48002A0E5E6E010E0101F36F2C0EF26F010E4B
:103C58000101F56F000E00019D6F020E00019E6FBD
:103C6800000E2A6E000E2C6E9DC0D9FF9EC0DAFF92
:103C7800000EDF6E000E00019C6F010E9B6F12009C
:103C8800E50E366E7E0E376E23EC21F00F0EC11254
:103C9800200E896E000E8B6E946893689268928AE3
:103CA800C70ED56EF294000E2A6E000E2C6E000E12
:103CB8002D6E0BD02D50010D400EF324D96E030E3E
:103CC800F420DA6E000EDF6E2D2A7F0E2D64F2D7F7
:103CD800000E2D6E0BD02D50010D420EF324D96E1F
:103CE800010EF420DA6E000EDF6E2D2A3F0E2D64D1
:103CF800F2D712000600E9CF52F0EACF53F0E1CF35
:103D080054F0E2CF55F0D9CF56F0DACF57F0F3CFD1
:103D180058F0F4CF59F0F6CF5AF0F7CF5BF0F8CF60
:103D28005CF0F5CF5DF020EC12F05DC0F5FF5CC0F3
:103D3800F8FF5BC0F7FF5AC0F6FF59C0F4FF58C040
:103D4800F3FF57C0DAFF56C0D9FF55C0E2FF54C091
:103D5800E1FF53C0EAFF52C0E9FF51C0FBFF50C06A
:103D6800FAFF5F921100000E0101DC6F4B0EDD6F50
:103D7800000EDE6F000EDF6F000E0101E06F000E17
:103D88000101E16F080E0101E26F000E246E1A0EA8
:103D98003C6E010ED6EC21F01E0E3C6E020ED6ECE7
:103DA80021F0000E346E400E356E050E366E400E54
:103DB800376E020E51EC14F034C028F135C029F1E9
:103DC800000E0101266F000E0101276F000E000191
:103DD800FD6F1200000EFEEC22F0000E0101416F93
:103DE800000E01013C6FA7EC22F0490E0001626F42
:103DF8007F0E0001636FF9EC20F0000E0001606F88
:103E0800020E0001616F000E0001636F000E626F09
:103E1800000E0001656F400E646F45EC22F0000E45
:103E28000101306F020E0101316F82EC0FF05FEC7F
:103E380022F0080E296E92EC1DF0C7EC0EF0FDD7AB
:103E48000001695100016A11D8B426D0010E0001A1
:103E58006B6F06D00001D89069376A3700016B2B69
:103E680000016AAFF7D7000169510001675D0001E1
:103E78006A5100016859D8A008D0000169510001B1
:103E8800675F00016A510001685B0001D8906A33DE
:103E9800693300016B2FE7D767C067F068C068F027
:103EA8001200F60E00019F1916E1010E0001A0197B
:103EB800D8A411D09DC06CF09EC06DF0C40E000156
:103EC8006E6F7F0E00016F6FFEC070F00001716BA6
:103ED8000DEC00F010D09FC066F0A0C067F052EC67
:103EE80015F0000166510001FE6F9DC0D9FF9EC00C
:103EF800DAFF000EDF6E000E00019C6F010E9B6F53
:103F08001200F60E00019F1916E1010E0001A0191A
:103F1800D8A411D09DC06CF09EC06DF0C40E0001F5
:103F28006E6F7F0E00016F6FF2C170F0F3C171F018
:103F38000DEC00F010D09FC066F0A0C067F052EC06
:103F480015F066C0F2F167C0F3F19DC0D9FF9EC0BD
:103F5800DAFF000EDF6E000E00019C6F010E9B6FF2
:103F68001200F60E00019F1916E1010E0001A019BA
:103F7800D8A411D09DC06CF09EC06DF0C40E000195
:103F88006E6F7F0E00016F6FF4C170F00001716BEE
:103F98000DEC00F010D09FC066F0A0C067F052ECA6
:103FA80015F0000166510101F46F9DC0D9FF9EC054
:103FB800DAFF000EDF6E000E00019C6F010E9B6F92
:103FC8001200F60E00019F1916E1010E0001A0195A
:103FD800D8A411D09DC06CF09EC06DF0C40E000135
:103FE8006E6F7F0E00016F6FFFC070F00001716B84
:103FF8000DEC00F010D09FC066F0A0C067F052EC46
:1040080015F0000166510001FF6F9DC0D9FF9EC0E9
:10401800DAFF000EDF6E000E00019C6F010E9B6F31
:104028001200020E2618D8A403D047EC13F0120091
:10403800000E266E01013551D8A41FD020EE01F0E4
:104048001B50D9261C50DA22080EDF6E20EE02F033
:104058001B50D9261C50DA22300EDE6E040EDD6E9F
:104068001BC0D9FF1CC0DAFF0C0EDF6E1BC0D9FFC6
:104078001CC0DAFF000EDB8E1200000E0101356F46
:104088001200F60E00019F1916E1010E0001A01999
:10409800D8A411D09DC06CF09EC06DF0C40E000174
:1040A8006E6F7F0E00016F6F5EC070F00001716B64
:1040B8000DEC00F00FD09FC066F0A0C067F052EC86
:1040C80015F0000166515E6E9DC0D9FF9EC0DAFFF3
:1040D800000EDF6E000E00019C6F010E9B6F120038
:1040E80092928092A00E156E860E166E010E176EB5
:1040F800000E186E05D01506000E165A175A185AD3
:104108001550161017101810D8A4F5D7928280826F
:10411800A00E156E860E166E010E176E000E186E26
:1041280005D01506000E165A175A185A15501610AB
:1041380017101810D8B41200F4D7BF7FCA3FB57F44
:104148008C39E87F0E33D87FFA38EC7F6A3F6A7F74
:104158008A40F07F6838BA7F7246C87FD846CC7FDD
:10416800BA46DC7FD637B07FE834317F0A3FAB7F71
:10417800BA31F47F143C7C7F28479F7F9A27E07FE1
:10418800E642D47F1E3AE47FEE44997FAA3ED07F70
:104198000000A09A0001FD51D8B402D0A08A1200F4
:1041A800000E0001646F60C062F061C063F000013E
:1041B800642B00016429D8B40AD062C0D9FF63C057
:1041C800DAFF0001624B632BDF50D8A4F0D760C040
:1041D80021F161C022F164C025F0010E01013D6F9B
:1041E800010E0001FD6FA08A120015D062C0F6FF13
:1041F80063C0F7FFF86A070EF76403D00800F550AC
:1042080005D0F6CFE1FFF7CFE2FFE750ACEC23F0A3
:104218000001624B632B62C0F6FF63C0F7FFF86AC8
:10422800070EF76403D00800F55005D0F6CFE1FF7C
:10423800F7CFE2FFE7500009D8B41200D7D714D05F
:1042480036C0F6FF37C0F7FFF86A070EF76403D0E9
:104258000800F55005D0F6CFE1FFF7CFE2FFE750B1
:10426800B7EC23F0364A372A36C0F6FF37C0F7FFD7
:10427800F86A070EF76403D00800F55005D0F6CFAA
:10428800E1FFF7CFE2FFE7500009D8B41200D8D712
:1042980060C064F061C065F003D00001644B652B19
:1042A80064C0F6FF65C0F7FF0800F5500009D8A400
:1042B800F4D760C062F061C063F00001621F631F41
:1042C800624B632B00016451000162250001606F9D
:1042D80000016551000163210001616F1200000EA9
:1042E8000001A26F010EA16F80A405D0000E00018D
:1042F800A26F000EA16F9DC06CF09EC06DF0C40E41
:1043080000016E6F7F0E00016F6FA1C070F0A2C038
:1043180071F00DEC00F0000E00019C6F010E9B6F18
:10432800120070A01DD019C0D9FF1AC0DAFF800E84
:10433800DE18D8A414D00FC0D9FF10C0DAFF840E3D
:10434800DE18D8A40CD019C0D9FF1AC0DAFF0C0E99
:10435800DF6E19C0D9FF1AC0DAFF000EDB8E70902D
:10436800689A120036C03CF037C03DF034C03AF0CD
:1043780035C03BF00ED03CC0D9FF3DC0DAFF3AC093
:10438800E1FF3BC0E2FFDFCFE7FF3C4A3D2A3A4A64
:104398003B2A3806D8A039063828EDE13928D8B4A0
:1043A8001200E9D73F6E3CA405D0000E346E3F5092
:1043B800A1EC1BF03CA205D0010E346E3F50A1ECDD
:1043C8001BF03F50010D700EF3243D6E0F0EF420CC
:1043D8003E6E3DC0D9FF3EC0DAFF3CC0DFFF120091
:1043E8000001656F010E0001646F7B0E00016561BD
:1043F80004D0610E0001656109D000016551D4EC5B
:1044080022F0D8B003D0000E0001646F64C063F0DE
:104418000001633112000001605100016203F3CF13
:1044280064F0F4CF65F00001605100016303F350BC
:10443800000165270001615100016203F35000018A
:10444800652764C060F065C061F01200000E0101CC
:10445800366F000E416E740E406E000E426E000EF6
:10446800436E000E456E000E446E51EC1DF06D92C9
:10447800699401D0689468B4FDD7000E01013B6FC0
:10448800120060C066F061C067F009D066C0D9FF4D
:1044980067C0DAFF62C0DFFF0001664B672B0001CF
:1044A8006407D8A0650700016429F0E100016529C7
:1044B800D8B41200EBD72150D8A41200000E6D6EAC
:1044C800000E696E160E6F6E9F0E6B6E7B0E696E18
:1044D800D08EA28AA08AF28E01D06D866DA6FDD7F5
:1044E800010E216E12009DC06CF09EC06DF01F0E73
:1044F80000016E6F7E0E00016F6F250E0001706F58
:104508007F0E0001716F0DEC00F0000E00019C6F32
:10451800010E9B6F1200698468986D82010E01017B
:10452800366F000E01013B6F000E416E750E406E36
:10453800000E426E000E436E000E456E000E446E75
:1045480051EC1DF012000C0EAF6E000EB06EB89656
:10455800AC98AB8EAB88AB9A9D989D9AD08E9F8A6B
:10456800F28EAC90AB9CAC9AAC8AAC94000E010174
:104578003F6F120034C03AF035C03BF008D03AC063
:10458800D9FF3BC0DAFF36C0DFFF3A4A3B2A38067C
:10459800D8A039063828F3E13928D8B41200EFD763
:1045A8000001626F000E0001616F5B0E0001626125
:1045B80007D0400E0001626503D0010E0001616F53
:1045C80061C060F00001603112000001626F000EEE
:1045D8000001616F3A0E0001626107D02F0E0001E1
:1045E800626503D0010E0001616F61C060F00001D7
:1045F800603112000001606F07D0010EC9EC23F092
:10460800010ECAEC23F0120000016051000AD8B470
:10461800F4D7010AD8B41200030A1200010E0101EE
:104628001427000E15231623172301013651D8A489
:10463800120001013B2B01013B51D8A412000101DA
:104648003B691200A09A0001FD51D8A40CD060C0AB
:1046580021F161C022F162C025F0010E01013D6F18
:10466800010E0001FD6FA08A12009DC06CF09EC073
:104678006DF0D80E00016E6F7D0E00016F6F0DECAE
:1046880000F0000E00019C6F010E9B6F1200346E4B
:1046980007D0010ECBEC23F0010ECCEC23F0120076
:1046A8003450000AD8B4F5D7010AD8B41200030A66
:1046B8001200000EA0EC23F09DC0D9FF9EC0DAFFC7
:1046C800000EDF6E000E00019C6F010E9B6F120042
:1046D80074EC20F09DC0D9FF9EC0DAFF000EDF6E9B
:1046E800000E00019C6F010E9B6F1200ABA204D05C
:1046F800AC9AAC8AAB98AB88ABA41200AECF60F092
:10470800AC9AAC8A1200ABA204D0AC9AAC8AAB9833
:10471800AB88ABA41200AECF34F0AC9AAC8A1200CE
:104728009DC0D9FF9EC0DAFF000EDF6E000E0001AB
:104738009C6F010E9B6F12000001606F0001600505
:10474800D8A403D0929A809A1200928A808A120082
:104758000001616F03D07AEC23F004009EA8FBD718
:1047680061C0ADFF1200356E03D087EC23F0040062
:104778009EA8FBD735C0ADFF12002C0103014E5592
:034788004C4C0096
:10478C0044EC1EF012001200120012001200120073
:04479C0012002A14C9
:107CF0000001000800400000020010008001000A9E
:107D0000006400E80310270100100000010010D4F7
:107D10007D5A7D8E7D177D09024300020100C0322D
:107D200009040000010202010005240010010424DE
:107D30000202052406000105240100010705810354
:107D400008000209040100020A00000007050202FF
:107D50004000000705820240000034034D00690026
:107D6000630072006F00630068006900700020000B
:107D700054006500630068006E006F006C006F00C7
:107D800067007900200049006E0063002E00340374
:107D90004300440043002000520053002D003200F5
:107DA00033003200200045006D0075006C0061005A
:107DB000740069006F006E002000440065006D00D3
:107DC0006F001201000202000008D8040A0000013E
:107DD00001020001040309044E6565642068656CB6
:107DE000703F204C6F6F6B20696E20746865207344
:107DF0006F7572636520636F6465210A0020677088
:107E000069625F7074723A20256420706F727461C9
:107E10003A2025582074726961733A20255800472A
:107E20005049422D55534220436F6E74726F6C6CF3
:107E300065722076657220362E342025730A000D77
:107E40000A53706F6C6C207374617475732062795F
:107E500074653A20255820000D0A636F6D6D616EC0
:107E6000643A202573202573206C656E20256420DC
:107E7000000D0A52583A2025642074696D656F75AB
:107E80007420256420000D0A64756D70696E67208A
:107E9000646174613A202573200030313233343507
:107EA0003637383941424344454600303132333465
:107EB00035363738396162636465660020657869F4
:107EC00074696E6720636C7220000D0A46726F6DD4
:107ED00020475049423A200020696E73696465204A
:107EE000636C722000475049425F496E69742829CB
:107EF00020000D0A54583A202558202558200043C8
:107F00004D44206C656E3A20256420000D0A4672AF
:107F10006F6D205553423A20000D0A646174613A36
:107F200020257320005365702032372032303136DF
:107F300000726561645F746D6F5F6D73005B253007
:107F400032585D3C454F493E005374617274696E0E
:107F5000672E2E2E007265706C793A2025732000F2
:107F60002074696D656F75742000656F745F636858
:107F700061720044415441206C656E007361766506
:107F800063666700286E756C6C29003C253032589A
:107F90003E005B253032585D006465627567007392
:107FA000706F6C6C003C4552523E0072656164001B
:107FB0006D6F6465006175746F0068656C70006159
:107FC0006464720025640A00696663006C6F630074
:107FD000656E640074726700656F69006C6F6E0097
:107FE0007372710076657200636C7200656F730066
:0F7FF000656F7400727374000D0A002563000042
:020000040020DA
:08000000FFFFFFFFFFFFFFFF00
:020000040030CA
:0E000000240E3F1EFF8181FF0FC00FE00F4056
:00000001FF
